:4000000000080020110000006B0100006B01000010B500F08FFE00F061F900F0AFF8000010B572B6EE22134B12021A60FF22124B124C1A60124BF33A1A609022114B120128
:400040001A603622104B18201A601123236000F0AFFDC0220D4BD2001A600D4A0D4B1A6004220D4B1A600D4B3C321A600023236010BDC046000102400003024030001040E6
:400080000001044008010440080304400003014040FF008000000140280003400001014000000000000000000000000000000000000000000000000000000000000000006E
:4000C0000000000000000000000000000000000000000000000000000000000000000000000000000000000000000000000000000000000000000000000000000000000000
:4001000010B5064C2378002B07D1054B002B02D0044800E000BF0123237010BDF8000020000000005C130000084B10B5002B03D00749084800E000BF07480368002B00D1BC
:4001400010BD064B002BFBD09847F9E700000000FC0000205C130000700000200000000010B562B600F0E8FAFEE710B501F0B4F803680C2B00D1FEE7FEE70000F8B500258C
:400180000F49104B01394A1C14D000221F685C689E68A018B24203D0B858A0500432F8E70200DE68141AA64201D020C2FAE710330139E8E701F096F8FFF7D2FFFEE7C04692
:4001C000010000009413000001210F4A70B5136814008B43136000230C4D0D4E0D489A002900032B00D8B15801338150192BF6D1FFF716FF084B1A68002A00D11A60012261
:4002000023681343236070BD000010406B010000000000000000002068000020004700234118002A05D0013A881800781B18DBB2F7E7180070470000013810B50B2831D80D
:400240008901494201F034F806090B0D0F111513171A1C21FF239B0113E0154B16E0154B0AE0154B12E0154B0BE0154B09E0154B02E0154B00E0154BC91814E0144B05E03D
:40028000144BC9180878C0B211E0134BC9180A7848788C780002230418430300C8781343000603E000210B7848780002184310BDC13F0000C53F0000C93F0000D03F0000E7
:4002C000D13F0000D63F0000D23F0000D43F0000D83F0000DC3F0000E03F00000C4B10B51A68102313400B4A00D113601368802B0DD10024022021001460FFF79DFFA04254
:4003000005D021000220FFF797FFFFF787FF10BD5400034068000020F8B5010006000320FFF78AFF040031000420FFF785FF0134A4012718002431000320FFF77DFF250060
:4003400001308001B84209D203785A1ED2B2FD2A00D80125E418E4B20130F3E731000120FFF76AFF6442E4B20623844203D16A4255416D422B401800F8BD0000F0B5C04C33
:40038000A544019000F032FA62B6019B002B02D06B461B7901E0BB4B1B78DBB2039300250A23009502939621039B04AA49000AA800F038FA019B002B03D0029B013BDBB278
:4003C0000293029B002B02D00028ECD102E0002800D08BE004AB1988062900D84BE11A7E0423012A52D104AA568BF21D8A4200D943E1962149008A4200D93EE10AAA92198A
:400400009279172A42D10022F3189BB2002B09D0A0A99D48C91809180978013B521892B29BB2F3E70AAFBB19597952421B79090292B219430823914228D162E0342B00D083
:40044000CAE0009B012B00D015E1032E00D012E14022002155A800F074FF40251F2155AB581904AB7519F21EC918ADB200F060FF432D00D0F9E004AB9D7F587F2D0205434A
:40048000FF2D00D810E1012300930933002404AA548001210AAA5370230AD370002311709470221D92B2002A09D0A0A97648891809180978013A5B189BB292B2F3E7A0AACA
:4004C000724912195B4251189BB20B7070491B0A51180B706F4B0734D2181723137004AAA1B27F3302320AA800F0D0F9019B002B00D158E7009B012B00D016E1012300937C
:4005000051E77B783C79180031380A282ED9624A1468002C26D0009A012A25D104AAD68007AE13710BAF0C2200213000069700F008FFB760310005A8A0472623B488FF337F
:400540009C4202D9B368BB4207D0B268002A01D1002C04D13368DBB299E70E2396E70E23140094E7052392E705238FE700F0AAFE0B001900CFFF66FF3A00CFFF3E005000E2
:4005800066FF60007000009B012B74D1002E72D13000FFF7C1FE43424341009C3B71330075E7009B012B66D1012E64D1002C62D13A4B1B681B689A0BD2B29B09DBB2002AF4
:4005C00001D080235B003B711B0A7B71FF23BB7100230424FB715AE7009B012B4BD1022E49D93BE7009B012B45D198E0009B012B41D12C337419FF339C423EDC55AB58191D
:4006000032000BA900F094FE0023A5B21C003EE7002E30D107AB1900214A350011CA11C10BAA03CB03C201230824009333002EE7009B012B1FD1032E1DD104AA04AB977F94
:400640005B7F3F021F430A23FF2F00D91EE748E00020FFF761FE002802D18022114B1A6000F0DCF800F044FB05E001230025009302332C000BE7042308E7032306E7C0467E
:400680007CFDFFFF60130000A7FDFFFFACFDFFFFADFDFFFFAEFDFFFF14010020740000206413000068000020224B1B681A6893099BB2920601D001339BB220022D18A8B2E8
:4006C000834204D90123002500930933D1E755A900F02AF90028F5D10123050000930300C7E72102C919890140220020FFF797FD0600002C0DD1FF2F0BD121000520FFF72B
:400700009BFD2100361A0620FFF796FDF6B2361AF6B20AAB76421E7101240023B7E60025019BAB4200D0E9E63DE6A1239B009D44F0BDC0467400002070B50020FFF7ECFD65
:40074000431E98410625144C4042236805401A68C021C03A0020FFF762FD63681B78181AC0B2834203D123681B68002B02D1002000F0BCFA094C2368402B01D0002D03D007
:4007800000202060FFF7FAFD1420FFF7F7FD8023236000F0ADFA70BD74000020680000200D4B1B685B0615D50C4B1B68DB0609D50B4B1A68002A0DD00A490A6000220A49B8
:4007C0000A6006E0084B074A18681168884201D012681A607047C0464C0F06406400064018010020C0010020B001002010B5094C4021201D00F07EF820000021443000F0C7
:400800005BF8054800F0E4FA0023236000F0BCFA10BDC04618010020A107000010B500F0C1FA10BDF7B506000D0001920120002E24D0002922D00A2410275C43002C1CD041
:400840000F4803783B4213D00E4A019913689BB20B800021017011602A1C9D4200D91A1C094992B20431300000F062FD002005E0012000F049FA013CE0E71020FEBDC04632
:40088000B8010020BC0100201801002070B501230C0000280CD000290AD0064D11802B0044330A000100180000F042FD00232C60180070BD1801002070B504000D0000288A
:4008C0000ED0052000F0FEF9064B074A1C60074B05201D6000231360054A136000F0E8F970BDC046CC010020B0010020C0010020B401002070B504000D0000280CD00520CD
:4009000000F0E0F90022054B05201C60044B1D60044B1A6000F0CCF970BDC046C8010020C4010020BC010020F0B500279DB0089703900997FF2800D9F2E0B94200D1EFE05B
:4009400040220CA800F0F4FC0222390001970AAB9000C058002802D00918074301920132122AF5D1002903D1002F00D0DBE000E0002702973F227149714C0A9171485A60C5
:40098000714A23600260C046236806911B0F049007920F2B04D022680023120F0A2A01D02368DBB20893089D002D00D0C2E000F0D5F9664E66493268664B0A601B68059052
:4009C000DB0FDB074B60644B1B6809959B00099818338B600D0000281ED1302B06D12D3B1A4203D112091A40012A13D0022000F02BF9AB68302B02D0302000F0D9F800F056
:400A0000B5F8002000F0C4F8302233689343203A1343336000230893089B002B18D14F4A03990A920A9A09040A430AA90A92049821604B49424A0160C0462168090F0F2927
:400A400003D01168090F0A2901D01368DBB20893089D002D3BD1002F39D0290040220CA800F06FFC019B029A0AAF9B00DA51069B049A0A933F2307997B602760304B1160D8
:400A8000C0462268120F0F2A03D01A68120F0A2A01D01D68EDB20895089B002B17D1314A03990A920A9A09040A4304982E490A922760234A0160C0462168090F0F2903D0F3
:400AC0001168090F0A2901D01368DBB20893099B002B21D11E4CA068302808D1226803331A4206D112091340012B02D10DE000F05FF803202368184000F04AF82368336070
:400B00006368002B01D100F03BF800230993099B002B01D0099B0893059800F023F909E00423089306E0019A012792009858995002901FE708981DB0F0BDC046B6D700007F
:400B4000080010400400104004000080280003409C01002030000340080F0340B6D8000005000080B6D90000060000808021034A090613680B4313607047C04630000340BF
:400B8000024A13685B005B08136070473000034010B5040000F0E2F8032304490A689A43234013430B6000F0DDF810BD28000340F8B50400182804D0102302009A43202A7C
:400BC00035D1072600F0CAF8194D1A4A2B681A49B3432B60194B0700E3181B78DBB21360174A1368B3431360164B0A68E31818787F239A43034013430B60322000F0A4F8D2
:400C0000182C11D923002A681C3B9B08B243334013432B60322000F097F8183C2B68A4083440B3431C432C60380000F09BF8F8BD080F03400C0F0340180F0340CDF1FF0F77
:400C4000100F0340B4F1FF0F10B5040000F086F8A3000C24044923400A68A24313430B6000F080F810BDC04628000340024B8000C31818681960704740000020F8B5032659
:400C800005003540B5400F0004000635AE40AF4000F064F8A408054BA400E4182368B3431F43276000F05EF8F8BDC04600E400E01F2318401E3B8340014A13607047C04652
:400CC00000E100E01F2318401E3B8340014A13607047C04680E100E01F2318401E3B8340014A13607047C04680E200E001BE7047034A044913689BB20B4313607047C046F8
:400D00000CED00E00400FA0570B5802504002D02064BAC4205D9586800F016F8044BE418F6E79868604300F00FF870BD7C0000200080FFFF014A024B1A6070476588EDACA7
:400D400038000340000000000230800804D0C0460138FDD1C046C046C0467047EFF3108072B6704780F310887047C0468021054A10B5136809060B4313600520FFF798FFC9
:400D800010BDC0460000064010B5054C2378002B03D100F041F801232370FFF7E7FF10BDA801002010B50520FFF78CFF00F096F8054A052013685B005B0813600022034B9F
:400DC0001A60FFF789FF10BD00000640880F0640014B58607047C046A801002080200A4B40001A6802420AD0084A1268520406D41A680749114019601A6802431A600222AF
:400E0000044B1A607047C0460000064060000640FFFEFFFF6C00064010B500241A4B1B4A1C601B4B1B491A601B4B1C4A052013601B4A14601B4A11601B4A13601B4B1C6053
:400E4000FFF740FF03210520FFF718FF18490520FFF70CFF4C22174BFF321C60164B1A60164B3C3A1C60164BFF3A1C60154B1C60154B1A70154B1C70154B1C60154B1C6035
:400E8000154B1C7010BDC0460000064088080040600006401200FE00070100800003064004030640100306400002064004020640590F0000880E0640480F0640080F06405E
:400EC000C80F0640880F0640D1010020B8010020B0010020BC010020D00100200023044A1360044A13601022034B1A707047C046680006406C000640D10100200E4A10B5B3
:400F000013680E495B005B08136000230B600C490C480B6004680C49214001600B490B600B490B6010210B4B19708021136809060B43136010BDC046000006406800064048
:400F40006C00064060000640FF5CFFFF880F0640C80F0640D1010020B24BF7B51B68002B00D09847B04B1B68DB0702D50022AF4B1A602020AE4B1A78024219D1AD4A116898
:400F80000222FF32114213D01978AB4AC90706D511781E38814311701178073004E0117881431170902110780143117000221A701A78920600D533E11A78D20600D42DE1D6
:400FC00002229C480168114234D09C499C4D0A609C490D320C68096822409B4C0904C90F26788A189449B24204D204260A7832430A7004E027782E68D21BB21A2A602D6847
:40100000924A15600022924D2A6080252270914C6D0222682A43226025688F4A2A40226002240A78A2430A700A78013C22430A7010221A7008220168114235D07F490A6008
:40104000864A1168890417D58549864F0F25864C24682C420CD06E460C683D682C19834D2D68F571F57925700C6801340C60EDE714687F49214011607E4A6F49156814003F
:40108000AA0603D540250A782A430A7000257A4A15607A4A226020240A78A2430A700A78103C22430A701C70026852063ED50121734A1160734A60491068102210420BD076
:4010C00063480260614A10685D4A106002200A7802430A7012221DE06B4A614812680068121A0420072A0ED95C48082A05D1A024026824022243026007E080240268A4010C
:401100002243026008205C4A106020200A7802430A70112208211A705C4A484B1A605C4A13680B43136001225A4B1A6008215A4B1A680A4225D0544B494A1B681068083B6B
:401140001B1A01208B4201D900200B00454C474D002B0AD011682668013B71182E68F6B20E70116801311160F2E7002807D080203A4900020A6802430A603F4A1360082235
:401180001FE01B685B071ED5384B35491A683E4B08681B6898420CD201203E4BD2B2186030480B680068C3181A700B6801330B6006E0FFF713FE40211F4A13780B4313701E
:4011C00004222C4B1A60354B1B68DB0628D50F21FF25334B1B481C68194A03680B40082B18D0304B17681B682F4E9F4208D21368E3181B78DBB23360136801331360ECE737
:401200003560114E33780A2BE7D833780133DBB23370E2E71022254B1A6001E0FFF76EFEF7BDC046AC0100208C0E0640880E0640D10100204C0F0640B8010020400F0640A0
:40124000B401002008020640D0010020B0010020880F064004020640FFFFFEFF60000640BC010020C80100200803064040030640FF5FFFFFC00F0640C80F0640ED0F000093
:40128000800E064064000640C4010020FF0F0000480F06406C000640CC0F06408C0F0640CC010020C001002040020640800F064002B4714649084900095C49008E4402BCFC
:4012C0007047C04603B47146490840004900095E49008E4403BC7047014B18687047C046F00000200E4B70B500251E000D4CE41AA410A54204D0AB00F35898470135F8E7E7
:4013000000F036F8084B00251E00084CE41AA410A54204D0AB00F35898470135F8E770BD7C1300007C1300007C13000084130000002310B59A4203D0CC5CC4540133F9E7F2
:4013400010BD03008218934202D019700133FAE77047000040140000C000000000000000FF0000009A11440A003C010143000000F8B5C046F8BC08BC9E467047290100008A
:40138000C9010000F8B5C046F8BC08BC9E46704701010000A81300007000002088000000E0000000000000000000000054130000581300000100000000007017E02E000080
:4013C0000C000000001BB70000000000000000000000000000000000000000000000000000000000000000006C130000000000000000000000000000000000000000000090
:4014000000000000000000000000000000000000000000000000000000000000000000000000000000000000900000200000000000000000000000000000000000000000FC
:401440000008002051140000D11F0000D11F000010B5034B83F3088800F0C4FE00F0C0FD0008002010B50E4C11232360182000F01FFE00230B4A13600B4A0C491160C0205E
:40148000C0000B4908600B49116004210A4A11603C310A4A11600131094A1160236010BD30001040000301400000014040FF00800403014041FF0080280003400C01014004
:4014C0000001014010B572B6EE2212020B4B1A60FF220B4B1A60E93A0A4B1A600A4A0B4B1A600C220A4B1A6090221201094B1A603622094B1A60FFF7B5FF10BD0001024052
:401500000003024000000440B061000008000440000104400801044008030440000000000000000000000000000000000000000000000000000000000000000000000000E4
:4015400010B5064C2378002B07D1054B002B02D0044800E000BF0123237010BD0801002000000000E8280000084B10B5002B03D00749084800E000BF07480368002B00D1B6
:4015800010BD064B002BFBD09847F9E7000000000C010020E828000070000020000000000A4B01221A700A4A11785970917999709188080AD870197151785971917899712D
:4015C000D278DA7117221A727047C0467400002024010020024B00221A725A729A72704724010020082827D88000144B1B589F46134B585C21E0124B59183423C85C1CE06E
:401600000F4B59186823C85C17E00E4B5918087F13E00C4B59185023C85C0EE00A4B591808790AE0084B59183823C85C05E0064B59186C23C85C00E000207047EC2800000F
:4016400064290000E4290000642A000010B50C4B5B78002B02D0FF22094B5A70084B9B78002B02D0FF22064B9A70054BDB78002B02D0FF22024BDA70FFF792FF10BDC04686
:4016800024010020F0B583B000900191954BDD7A002D05D01A006B4603CB03C200251EE16B461C78072C00D1AEE00BD8032C58D003D8012C2DD01BD945E0052C00D17AE0A5
:4016C00064D993E00B2C00D1D6E005D8092C00D1B6E000D8A6E0C1E00D2C00D1E8E000D2D8E0FE2C00D1F1E0FF2C00D1F3E0F5E07C4D6B46280006CB06C0691C032201F064
:40170000E9F80023EB60AB80AB71FFF749FF2500E5E0744C6B46260006CB06C60027A771FA239B00A380FFF791FFE7602774022363742F33A374303BE374611C032230002C
:4017400001F0C8F8CBE0674C6B46220003CB03C20026E660A671FFF723FFFFF73BFFE674BDE0604C6B46260006CB06C60027A771FFF716FFE760E7743388A382B378A37503
:40178000611C0322300001F0A5F8A8E0554C6B46260006CB06C60027A771FFF701FFE760E7743388A382B378A375611C0322300001F090F893E04B4B6A46190011CA11C168
:4017C0009B79002B02D10822464B9A71454CFA23DB00A380FFF73AFF0023E360237404226274A374E374FFF7F5FE78E03D4B6A46190011CA11C10022DA60DA743A4B1A8ABD
:401800000A809B7C8B706AE0364B6A46190011CA11C10022DA60DA74334B9A8A0A809B7D8B705CE02F4B6A46190011CA11C10022DA60DA742C4B1A8A0A809B7C8B704EE027
:40184000284B6A46190011CA11C10022DA60DA74254B1A8B0A809B7E8B7040E0214B6A46190011CA11C10022DA60DA741E4B9A8B0A809B7F8B7032E01A4B6A46190011CA2E
:4018800011C10022DA60DA74174B1A8A0A809B7C8B7024E0134B6A46190011CA11C10022DA60DA74104B9A8B0A809B7F8B7016E00C4B6A46190011CA11C10022DA60DA74FC
:4018C000094B1A8B0A809B7E8B7008E000F0BAFF00F07CFC03E000F079FC00E0FF25280003B0F0BD240100207400002010B5334BDB7A022B15D0DAB2022A02D8012B05D06E
:401900003EE0032B1FD0042B2FD039E02B4AD37D0133DBB2D3752A49CB186C215B5C13723EE02649CA7D013AD2B2CA75244C6C20A218135C0B720A7E0132D3B20B76E31808
:401940001B5C4B722CE01D490A7E013AD2B20A761B4C6C20A218135C4B724A7E0132D3B24B76E3181B5C8B721AE0144A537E013BDBB253761249CB186C215B5C93720FE040
:401980000E4B0022DA729A76DA751A765A769A8B1A819A7F9A7218685968FFF773FE0CE0064A937E0133DBB29376302B05D9130000229A76DA7A0132DA7210BD240100209A
:4019C000642A000010B5C44AD3680A33D360D27A002A02D0FFF78AFF37E2BF4A12780D2A00D932E29200BD498A589746BA490023CB60080008300131032200F06BFF24E2A5
:401A0000B54A137C0133DBB21374527C934200D21BE2B14B00221A745B78002B04D0AE4B9A7CAF498A5C1A72AB4B9B78002B04D0A94B9A7CAA498A5C5A72A74BDB78002B40
:401A400004D0A54B9A7CA6498A5C9A72A24BDB7C002B0BD1A04B9B7C302B03D901229E4BDA74F2E101339C4A9374EEE19A4B9B7C002B04D1984B0022DA749A74E5E1013BAB
:401A8000954A9374E1E1944A9288934200D2DCE1914B0022DA60DB7C002B09D18E490133CB74080008300131033200F013FFCCE10022894BDA74FFF78DFDC6E1864AD27C65
:401AC000002A00D0C1E1844A9288934200D2BCE1814B9A8A1A819A7D9A720122DA74B4E17D4AD27C002A0BD17B4989888B4207D3794B0132DA740022DA60FFF76BFD0EE0E6
:401B0000012A0CD1F92B0AD973490132CA740023CB60080008300131013200F0DBFE6E4BDB7C022B00D090E16B4A9188D268914200D98AE1684A0133D374938A1381937D22
:401B4000937282E1644A137C0133DBB21374527C934200D279E1604B00221A745B78002B05D05D4CA17CA079FFF73CFD20725A4B9B78002B05D0584CA17CA079FFF732FD24
:401B80006072554BDB78002B05D0534CA17CA079FFF728FDA072504BDB7C002B0BD14E4B9B7C302B03D901224B4BDA744DE10133494A937449E1484B9B7C002B04D1464B16
:401BC0000022DA749A7440E1013B434A93743CE1414A9288934200D237E13F4A0023D360D37C0133DBB2D374012B0BD0002B02D0022B0ED014E0384B3A4A118A1981927C72
:401C00009A7222E1344B374A918B1981927F9A721BE1314B334A118B1981927E9A7214E12D4B0022DA742F4A118A1981927C9A720BE1294A9288934200D206E1264A00233C
:401C4000D360D37C0133DBB2D374062B3AD89B00254AD3589F46204B224A918A1981927D9A72F2E01C4B1F4A11002031128C1A818A789A72E9E0184B1A4A118B1981927EB5
:401C80009A72E2E0144B174A918B1981927F9A72DBE0114B134A11002431928C1A818A789A72D2E00C4B0F4A11002831128D1A818A789A72C9E0084B0A4A118A1981927C7B
:401CC0009A72C2E0044B0022DA74064A918A1981927D9A72B9E0C0462401002010290000042B00007400002048290000574A9288934200D2A9E0554B0022DA60DB7C002B9D
:401D000008D1524B0132DA74514A118A1981927C9A729AE04D4B0022DA744D4A918B1981927F9A7291E0494A9288934200D28CE0464B0022DA60DB7C002B08D1434B01329C
:401D4000DA74434A118B1981927E9A727DE03F4B0022DA743E4A118A1981927C9A7274E03A4A9288934270D3384B0022DA60DB7C002B08D1354B0132DA74354A918B19818E
:401D8000927F9A7261E0314B0022DA74304A118B1981927E9A7258E02C4A9288934254D32A4B0022DA60DB7C002B08D1274B0132DA74274A118A1981927C9A7245E0234BD7
:401DC0000022DA74224A11002C31928D1A818A789A723AE01D4A9288934236D31B4B0022DA60DB7C002B08D1184B0132DA74184A918B1981927F9A7227E0144B0022DA744C
:401E0000134A11002C31928D1A818A789A721CE00E4A9288934218D30C4B0022DA60DB7C002B08D1094B0132DA74094A118B1981927E9A7209E0054B0022DA74044A110051
:401E40002C31928D1A818A789A7210BD240100207400002010B5012000F0EEFC324B1B7A002B03D1002000F049FC12E0FF2B03D1012000F043FC0CE02B4AD27F002A03D181
:401E8000012000F03BFC04E0934202D8002000F035FC254B5B7A002B03D1002000F022FC12E0FF2B03D1012000F01CFC0CE01E4AD27F002A03D1012000F014FC04E09342FE
:401EC00002D8002000F00EFC174B9B7A002B03D1002000F08FF912E0FF2B03D1012000F089F90CE0104AD27F002A03D1012000F081F904E0934202D8002000F07BF90A4AD2
:401F0000D37F0133DBB2D377FF2B0BD113000022DA779B88002B03D1034BDB7A002B01D0FFF750FD10BDC0462401002030B585B0244B00229A76DA751A765A760132DA72B3
:401F4000214A09210D2000F021FA00F083F91F4800F006FC62B6FFF73DFBFF2000F056F9012000F069FC00F057FC00F0FDF90307FBD5154B1B78012B03D1134B1B7A172B8A
:401F800003D0FF22104B5A72EFE70F4C637802AD2B70A378AB71E37822791B021343AB80637901A90B70A3794B70E3798B7003220920684400F08EFC02986968FFF762FB84
:401FC0006072D2E72401002074000020551E000010B500F053FC03680C2B00D1FEE7FEE770B50F4E0F4D13E029686B68AC68002202E001C901C30432A242FAD1E868002297
:4020000002E0002102C304328242FAD11035013E002EE9D100F038FCFFF788FFFEE7C046010000005C2B000010B5114A136801218B43136000230AE0032B03D89A000D498F
:40204000505800E00C4899000C4A88500133182BF2D9FFF737FA0A4B1B68002B02D10022074B1A60024A116801230B43136010BD0000104040140000D11F00000000002065
:40208000680000201F2318401E3B8340014A13607047C04600E100E01F2318401E3B8340014A13607047C04680E100E001BE7047F8B50400182803D0202801D030283CD17C
:4020C00000F0D4FB05001F4A136807218B4313601D4BE3181B78DBB21C4A13601C4A13688B4313601B4803687F22934319001A4BE3181B7813400B430360322000F0ACFB13
:40210000182C16D90F4E33680727BB431A0023001C3B9B083B4013433360322000F09CFB3268BA432300183B9B083C001C4014433460280000F09EFB02E00020FFF7B6FF43
:40214000F8BDC046080F0340CDF1FF0F0C0F0340100F0340180F0340B4F1FF0F70B504000D00082802D90020FFF7A0FF1034A40080239B059C4664442068256070BDC046B6
:4021800070B504000E00032902D90020FFF78EFF082C02D90020FFF789FF03252540ED00063500F063FBA408A400074B9C46644421680323AB4099430B003100A94019436B
:4021C000216000F057FB70BD00E400E0034A13681B041B0C02490B43136070470CED00E00400FA05014A024B1A6070476588EDAC3800034004490A68D2B210239A43000160
:40220000184010430860704700000440044B1B68002BFBDB0002034B1843014B18607047000001404000008010B50520FFF72AFF10BDC04610B500F03BF810BD10B5044AF2
:402240001368802109060B431360FFF7EDFF10BD0000064010B5064B1B78002B04D1FFF7E9FF0122024B1A70FFF7E8FF10BDC046480100200A4B1B68DB050DD5094B1B6872
:402280005B0409D4064B1968074A0A401A601A68802149000A431A600222044B1A6070470000064060000640FFFEFFFF6C00064010B50024184B1C60184A194B1A60194B1F
:4022C000194A1360194A146019491A4A11601A4A13601A4B1C600520FFF7DEFE03210520FFF74EFF16490520FFF738FF154B1C605222FF32144B1A60144B1C60144B1C60FE
:40230000144B1C60144B1C70144B1C70144B1C80144B00221A7010BD0000064000080040600006400701008000030640040306401000FE00100306400002064004020640CC
:40234000BD230000880E0640480F0640080F0640C80F0640880F06405601002055010020600100205401002010B50520FFF794FE054B1C78E4B21A781F218A431A70052090
:40238000FFF780FE200010BD5501002070B506000D00141E0BD00520FFF77EFE044B1C60044B1E80044B1D800520FFF76BFE70BD580100205C0100205E01002070B5AA4B86
:4023C0001B68002B00D09847A84B1C88A84B1D68A84B1E680223FF331D4238D0A64A13685B005B081360A54A137820218B431370117810230B43DBB21370A14B1B68DB0628
:402400000CD4A04B1A78994B1B889A420CD09B4A117808230B43DBB2137005E0974A117802230B43DBB21370974A1168974B0B4013600023964A1360914A1360954A137017
:402440008D4A1368802109060B43136008E1F30602D50022904B1A600A23334200D190E08E4B1B685B0756D58D4B1B68894A1278002A16D0012A47D18A4A1288002A0DD01D
:402480000121894A1160894A12681219DBB213700134844A1388013B138038E0FFF7EAFE35E0834A128893422BD201217E4A1160804A1288934202D2D21A92B200E00022E3
:4024C00078490A80072A03D80121724A117014E0082A09D16C490A68A020000202430A6000216B4A116008E067490A688020800102430A600821664A1160624A13701C00D8
:4025000005E0FFF7B7FE02E00020FFF7CFFD0422694B1A6035E05C4B1B689B0431D5B3070DD5664B1B680F211940574A1068574B03401360012014E00821012011E0594B51
:402540001988083989B219800829F5D8002008E0564B1B681B19524A1268D2B21A70013401390029F4D1002808D1474A1368802109020B4313600022454B1A600C224E4B59
:402580001A60B3074BD5EB0615D50023404A13603B4A13603B4B1B789C4201D1022300E00A232B40354A11780B4320218B4313700022384B1A706B062FD5304A117820239C
:4025C0000B43DBB213702F4B1B781C003C4A1268D20612D5364A1288D31A324A1380394B1A68802149020A431A601968364A0A401A601022224B1A6002E00422244B1A60F7
:402600000122324B1A603249194B196031490868102303430B60244B1A60154B1D60154B1B685B071CD51F4B1B88002B0CD01F4B1B681B191B78DBB2274A13600134194A8D
:402640001388013B138002E0FF22234B1A60234B1B680F221340082BE5D10132204B1A60024B1C8070BDC0464C01002060010020400F0640000E06400000064055010020E0
:40268000880F06405401002060000640FF5FFFFFC80F064056010020880E0640CC0F064040030640500100206C000640580100205C0100205E010020C00F064008030640AE
:4026C0006400064004020640FFFFFEFF800E0640FF0F0000480F06404002064008020640800F064004490A68D2B204239A43800018401043086070470000044004490A6829
:40270000D2B202239A434000184010430860704700000440014B18667047C0460000002010B5040000F0A2F8044A1368C0218B43A4011C43146000F09DF810BD08E400E0BD
:4027400080225200014B1A607047C04600E100E080225200014B1A607047C04680E100E010B50400FFF7F4FF2000FFF7D3FF0320FFF7D6FFFFF7E4FF10BDC0460004000C25
:40278000014B18607047C046080105400004000C014B18607047C0461401054070B504000D0000F063F8AC40024B1C6000F062F870BDC0460800054010B500F057F8064A0B
:4027C000116801230B43136000F054F818210120FFF7E4FF10BDC04600000540014B18607047C0463801054010B580229204084B1A600D22074B1A600120FFF7EFFFEB2020
:402800004000FFF7C3FF0020FFF7B8FF10BDC046000105402401054010B5064B1B78002B04D1FFF7E1FF0122024B1A70FFF7C4FF10BDC04652010020014B18607047C04657
:402840003001054010B54022024B1A60FFF7BEFC10BDC046680000200230800804D0C0460138FDD1C046C046C0467047EFF3108072B6704780F310887047C046014B1868A0
:402880007047C046040100200E4B70B500251E000D4CE41AA410A54204D0AB00F35898470135F8E700F048F9084B00251E00084CE41AA410A54204D0AB00F3589847013532
:4028C000F8E770BD442B0000442B0000442B00004C2B0000002310B59A4203D0CC5CC4540133F9E710BD00000000000038160000F0150000F6150000001600000A160000BC
:40290000121600001C160000241600002E160000EC190000001A0000861A0000BC1A0000E01A0000441B0000D01B0000321C0000EC1C0000261D0000601D0000981D00001B
:40294000D41D0000101E0000561C0000641C0000761C0000841C0000921C0000A41C0000B61C000000050A10151A1F242A2F34393E44494E53585E63686D72787D82878D26
:4029800092979CA1A7ACB1B6BBC1C6CBD0D5DBE0E5EAEFF5FAFF0000000000010203040507090B0D0F1215181B1F22262A2F33383D42484D535960666D747B828A9199A259
:4029C000AAB3BBC4CED7E1EBF5FF0000000A141E28313B444C555D666E757D848B92999FA6ACB2B7BDC2C7CCD0D5D9DDE0E4E7EAEDF0F2F4F6F8FAFBFCFDFEFFFFFF00008E
:402A0000000001020305080A0E11151A1F242A30363D454D555E67707A858F98A1AAB2BAC2C9CFD5DBE0E5EAEEF1F5F7FAFCFDFEFFFF0000000000000000000101020203A6
:402A400004050607090B0D0F1114171A1E22262B30353B41474E555D656E77818B95A1ACB9C6D3E1F0FF0000000F1E2C3946535E6A747E88919AA2AAB1B8BEC4CACFD4D992
:402A8000DDE1E5E8EBEEF0F2F4F6F8F9FAFBFCFDFDFEFEFFFFFFFFFFFFFF000000000000010102030406090C0F13181D242B333B45505C69788796A3AFBAC4CCD4DBE2E7D8
:402AC000ECF0F3F6F9FBFCFDFEFEFFFFFFFF00000000010102020303050607090C0F13181D242E37424F5C6D7C8C9AABB8C4CED6DFE5EAEEF2F5F7F9FAFBFCFDFDFEFEFEFA
:402B0000FEFF0000FFFDFBF8F5F0EBE5DED6CDC4BAB1A8A099938E89868381817F7F7F808285898D9399A0A7B0B9C4CDD6DDE4EAF0F4F8FBFDFF4300F8B5C046F8BC08BC65
:402B40009E4670476915000029200000F8B5C046F8BC08BC9E46704741150000702B0000700000209800000060000000000000000000000001000000000000001700010497
:402B800001000000FF0000009400D3000000FF0000FF00004B008200FFFF0000FF7F0000FFFFFF00000000000000000000000000000000000000000000000000000000006A
:402BC00000000000362B0000000000000000000000000000000000000000000000000000000000000000000000000000000000000000000000000000000000000000000074
:402C000000000000A40000200000000000000000000000000000000000000000000000000000000000000000000000000000000000000000000000000000000000000000D0
:402C40000000000000000000000000000000000000000000000000000000000000000000000000000000000000000000000000000000000000000000000000000000000054
:402C80000000000000000000000000000000000000000000000000000000000000000000000000000000000000000000000000000000000000000000000000000000000014
:402CC00000000000000000000000000000000000000000000000000000000000000000000000000000000000000000000000000000000000000000000000000000000000D4
:402D00000000000000000000000000000000000000000000000000000000000000000000000000000000000000000000000000000000000000000000000000000000000093
:403FC0006D51140000500000000018000000000000000000000000000000000000000000000000000000000000000000000000000000000000000000000000000000000087
:0200000490303A
:020000004ED1DF
:0200000490402A
:200000000000000000000000000000000000000000000000000000000000000000000000E0
:0200000490501A
:0C00000000020A44119A00010A52606BD1
:0200000490600A
:0100000001FE
:00000001FF
